 Heap

 Timestamp is 2d9bfd4a (reproducible build file hash)

 Preferred load address is 0000000180000000

 Start         Length     Name                   Class
 0001:00000000 00003300H .text$mn                CODE
 0001:00003300 00000036H .text$mn$00             CODE
 0001:00003336 00000092H .text$x                 CODE
 0002:00000000 000001a8H .idata$5                DATA
 0002:000001a8 00000038H .00cfg                  DATA
 0002:000001e0 00000008H .CRT$XCA                DATA
 0002:000001e8 00000008H .CRT$XCZ                DATA
 0002:000001f0 00000008H .CRT$XIA                DATA
 0002:000001f8 00000008H .CRT$XIC                DATA
 0002:00000200 00000008H .CRT$XIZ                DATA
 0002:00000208 00000008H .CRT$XLA                DATA
 0002:00000210 00000008H .CRT$XLZ                DATA
 0002:00000218 00000008H .CRT$XPA                DATA
 0002:00000220 00000008H .CRT$XPZ                DATA
 0002:00000228 00000008H .CRT$XTA                DATA
 0002:00000230 00000010H .CRT$XTZ                DATA
 0002:00000238 00000000H .gehcont$y              DATA
 0002:00000238 00000000H .gfids$y                DATA
 0002:00000240 00001d40H .rdata                  DATA
 0002:00001f80 00000000H .rdata$CastGuardVftablesA DATA
 0002:00001f80 00000000H .rdata$CastGuardVftablesC DATA
 0002:00001f80 00000028H .rdata$T                DATA
 0002:00001fa8 000000a4H .rdata$voltmd           DATA
 0002:0000204c 00000314H .rdata$zzzdbg           DATA
 0002:00002360 00000008H .rtc$IAA                DATA
 0002:00002368 00000008H .rtc$IZZ                DATA
 0002:00002370 00000008H .rtc$TAA                DATA
 0002:00002378 00000008H .rtc$TZZ                DATA
 0002:00002380 00000004H .tls                    DATA
 0002:00002384 00000004H .tls$                   DATA
 0002:00002388 00000008H .tls$ZZZ                DATA
 0002:00002390 00000310H .xdata                  DATA
 0002:000026a0 00000898H .edata                  DATA
 0002:00002f38 00000078H .idata$2                DATA
 0002:00002fb0 00000018H .idata$3                DATA
 0002:00002fc8 000001a8H .idata$4                DATA
 0002:00003170 00000446H .idata$6                DATA
 0003:00000000 00000080H .data                   DATA
 0003:00000080 0001b268H .bss                    DATA
 0004:00000000 0000042cH .pdata                  DATA

  Address         Publics by Value              Rva+Base               Lib:Object

 0000:00000000       __AbsoluteZero             0000000000000000     <absolute>
 0000:00000000       ___safe_se_handler_count   0000000000000000     <absolute>
 0000:00000000       ___safe_se_handler_table   0000000000000000     <absolute>
 0000:00000000       __arm64x_extra_rfe_table   0000000000000000     <absolute>
 0000:00000000       __arm64x_extra_rfe_table_size 0000000000000000     <absolute>
 0000:00000000       __arm64x_native_entrypoint 0000000000000000     <absolute>
 0000:00000000       __arm64x_redirection_metadata 0000000000000000     <absolute>
 0000:00000000       __arm64x_redirection_metadata_count 0000000000000000     <absolute>
 0000:00000000       __dynamic_value_reloc_table 0000000000000000     <absolute>
 0000:00000000       __enclave_config           0000000000000000     <absolute>
 0000:00000000       __guard_check_icall_a64n_fptr 0000000000000000     <absolute>
 0000:00000000       __guard_eh_cont_count      0000000000000000     <absolute>
 0000:00000000       __guard_eh_cont_table      0000000000000000     <absolute>
 0000:00000000       __guard_fids_count         0000000000000000     <absolute>
 0000:00000000       __guard_fids_table         0000000000000000     <absolute>
 0000:00000000       __guard_iat_count          0000000000000000     <absolute>
 0000:00000000       __guard_iat_table          0000000000000000     <absolute>
 0000:00000000       __guard_longjmp_count      0000000000000000     <absolute>
 0000:00000000       __guard_longjmp_table      0000000000000000     <absolute>
 0000:00000000       __hybrid_auxiliary_iat     0000000000000000     <absolute>
 0000:00000000       __hybrid_auxiliary_iat_copy 0000000000000000     <absolute>
 0000:00000000       __hybrid_code_map          0000000000000000     <absolute>
 0000:00000000       __hybrid_code_map_count    0000000000000000     <absolute>
 0000:00000000       __x64_code_ranges_to_entry_points 0000000000000000     <absolute>
 0000:00000000       __x64_code_ranges_to_entry_points_count 0000000000000000     <absolute>
 0000:00000100       __guard_flags              0000000000000100     <absolute>
 0000:00000000       __ImageBase                0000000180000000     <linker-defined>
 0001:00000044       ?NewObject@JNIEnv_@@QEAAPEAV_jobject@@PEAV_jclass@@PEAU_jmethodID@@ZZ 0000000180001044 f i libHeap.obj
 0001:0000006c       ?SetEventNotificationMode@_jvmtiEnv@@QEAA?AW4jvmtiError@@W4jvmtiEventMode@@W4jvmtiEvent@@PEAV_jobject@@ZZ 000000018000106c f i libHeap.obj
 0001:00000078       ?TranslateError@@YAPEBDW4jvmtiError@@@Z 0000000180001078 f   libHeap.obj
 0001:00000330       ?nsk_jni_check_exception@@YAHPEAUJNIEnv_@@QEBDH@Z 0000000180001330 f   libHeap.obj
 0001:00000474       ?nsk_jni_lverify@@YAHHPEAUJNIEnv_@@HQEBDH1ZZ 0000000180001474 f   libHeap.obj
 0001:00000514       Agent_Initialize           0000000180001514 f   libHeap.obj
 0001:000006a4       Agent_OnAttach             00000001800016a4 f   libHeap.obj
 0001:000006a4       Agent_OnLoad               00000001800016a4 f   libHeap.obj
 0001:000006ac       Java_nsk_jvmti_unit_FollowReferences_FollowRefObjects_addRefToVerify 00000001800016ac f   libHeap.obj
 0001:00000884       Java_nsk_jvmti_unit_FollowReferences_FollowRefObjects_getTag 0000000180001884 f   libHeap.obj
 0001:00000944       Java_nsk_jvmti_unit_FollowReferences_FollowRefObjects_resetRefsToVerify 0000000180001944 f   libHeap.obj
 0001:0000094c       Java_nsk_jvmti_unit_FollowReferences_FollowRefObjects_resetTags 000000018000194c f   libHeap.obj
 0001:00000990       Java_nsk_jvmti_unit_FollowReferences_FollowRefObjects_setTag 0000000180001990 f   libHeap.obj
 0001:00000be8       Java_nsk_share_jvmti_ArgumentHandler_getAgentOptionsString 0000000180001be8 f   libHeap.obj
 0001:00000c98       Java_nsk_share_jvmti_DebugeeClass_checkStatus 0000000180001c98 f   libHeap.obj
 0001:00000d20       Java_nsk_share_jvmti_DebugeeClass_resetAgentData 0000000180001d20 f   libHeap.obj
 0001:00000d80       Java_nsk_share_jvmti_RedefineAgent_agentStatus 0000000180001d80 f   libHeap.obj
 0001:00000d8c       Java_nsk_share_jvmti_RedefineAgent_isRedefined 0000000180001d8c f   libHeap.obj
 0001:00000d98       Java_nsk_share_jvmti_RedefineAgent_redefineAttempted 0000000180001d98 f   libHeap.obj
 0001:00000da4       Java_nsk_share_jvmti_unit_Heap_getObjectCount 0000000180001da4 f   libHeap.obj
 0001:00000dac       Java_nsk_share_jvmti_unit_Heap_getObjectFreeCount 0000000180001dac f   libHeap.obj
 0001:00000db4       Java_nsk_share_jvmti_unit_Heap_getObjectSize 0000000180001db4 f   libHeap.obj
 0001:00000e08       Java_nsk_share_jvmti_unit_Heap_getObjectsWithTags 0000000180001e08 f   libHeap.obj
 0001:00001000       Java_nsk_share_jvmti_unit_Heap_getTag0 0000000180002000 f   libHeap.obj
 0001:00001054       Java_nsk_share_jvmti_unit_Heap_iterateOverHeap0 0000000180002054 f   libHeap.obj
 0001:000010bc       Java_nsk_share_jvmti_unit_Heap_iterateOverInstancesOfClass0 00000001800020bc f   libHeap.obj
 0001:00001138       Java_nsk_share_jvmti_unit_Heap_iterateOverObjectsReachableFromObject0 0000000180002138 f   libHeap.obj
 0001:00001198       Java_nsk_share_jvmti_unit_Heap_iterateOverReachableObjects0 0000000180002198 f   libHeap.obj
 0001:00001208       Java_nsk_share_jvmti_unit_Heap_newGlobalRef 0000000180002208 f   libHeap.obj
 0001:00001218       Java_nsk_share_jvmti_unit_Heap_objectResults 0000000180002218 f   libHeap.obj
 0001:00001220       Java_nsk_share_jvmti_unit_Heap_setHeapRootCallback 0000000180002220 f   libHeap.obj
 0001:00001240       Java_nsk_share_jvmti_unit_Heap_setKlassTagTestCallback 0000000180002240 f   libHeap.obj
 0001:00001250       Java_nsk_share_jvmti_unit_Heap_setObjectFreeCallback 0000000180002250 f   libHeap.obj
 0001:00001268       Java_nsk_share_jvmti_unit_Heap_setObjectRefCallback 0000000180002268 f   libHeap.obj
 0001:00001288       Java_nsk_share_jvmti_unit_Heap_setStackRefCallback 0000000180002288 f   libHeap.obj
 0001:000012a8       Java_nsk_share_jvmti_unit_Heap_setTag0 00000001800022a8 f   libHeap.obj
 0001:000012c4       Java_nsk_share_jvmti_unit_Heap_setTaggedObjectCountCallback 00000001800022c4 f   libHeap.obj
 0001:000012dc       Java_nsk_share_jvmti_unit_Heap_setTotalObjectCountCallback 00000001800022dc f   libHeap.obj
 0001:000012f4       Java_nsk_share_jvmti_unit_Heap_tagResults 00000001800022f4 f   libHeap.obj
 0001:000012fc       Java_nsk_share_jvmti_unit_Heap_zeroObjectCount 00000001800022fc f   libHeap.obj
 0001:00001304       Java_nsk_share_jvmti_unit_Heap_zeroObjectFreeCount 0000000180002304 f   libHeap.obj
 0001:0000130c       MA_checkStatus             000000018000230c f   libHeap.obj
 0001:000013b0       __local_stdio_printf_options 00000001800023b0 f i libHeap.obj
 0001:000015a8       exitOnError                00000001800025a8 f   libHeap.obj
 0001:0000165c       fprintf                    000000018000265c f i libHeap.obj
 0001:00001700       nsk_jvmti_lverify          0000000180002700 f   libHeap.obj
 0001:000017f0       nsk_jvmti_resetAgentData   00000001800027f0 f   libHeap.obj
 0001:00001870       nsk_jvmti_setFailStatus    0000000180002870 f   libHeap.obj
 0001:000018ac       nsk_lcomplain              00000001800028ac f   libHeap.obj
 0001:000018cc       nsk_ldisplay               00000001800028cc f   libHeap.obj
 0001:000018ec       nsk_ltrace                 00000001800028ec f   libHeap.obj
 0001:0000190c       nsk_lvcomplain             000000018000290c f   libHeap.obj
 0001:00001ac4       nsk_lvdisplay              0000000180002ac4 f   libHeap.obj
 0001:00001b10       nsk_lverify                0000000180002b10 f   libHeap.obj
 0001:00001b6c       nsk_lvtrace                0000000180002b6c f   libHeap.obj
 0001:00001bcc       nsk_printf                 0000000180002bcc f   libHeap.obj
 0001:00001bf4       nsk_vprintf                0000000180002bf4 f   libHeap.obj
 0001:00001cd4       printf                     0000000180002cd4 f i libHeap.obj
 0001:000023d8       __raise_securityfailure    00000001800033d8 f   MSVCRT:gs_report.obj
 0001:0000240c       __report_gsfailure         000000018000340c f   MSVCRT:gs_report.obj
 0001:0000264c       __GSHandlerCheck           000000018000364c f   MSVCRT:gshandler.obj
 0001:0000266c       __GSHandlerCheckCommon     000000018000366c f   MSVCRT:gshandler.obj
 0001:000026e0       __security_check_cookie    00000001800036e0 f   MSVCRT:amdsecgs.obj
 0001:00002a20       _DllMainCRTStartup         0000000180003a20 f   MSVCRT:dll_dllmain.obj
 0001:00002a60       __scrt_acquire_startup_lock 0000000180003a60 f   MSVCRT:utility.obj
 0001:00002a9c       __scrt_dllmain_after_initialize_c 0000000180003a9c f   MSVCRT:utility.obj
 0001:00002ad0       __scrt_dllmain_before_initialize_c 0000000180003ad0 f   MSVCRT:utility.obj
 0001:00002ae8       __scrt_dllmain_crt_thread_attach 0000000180003ae8 f   MSVCRT:utility.obj
 0001:00002b10       __scrt_dllmain_crt_thread_detach 0000000180003b10 f   MSVCRT:utility.obj
 0001:00002b28       __scrt_dllmain_exception_filter 0000000180003b28 f   MSVCRT:utility.obj
 0001:00002b88       __scrt_dllmain_uninitialize_c 0000000180003b88 f   MSVCRT:utility.obj
 0001:00002bb8       __scrt_dllmain_uninitialize_critical 0000000180003bb8 f   MSVCRT:utility.obj
 0001:00002bcc       __scrt_initialize_crt      0000000180003bcc f   MSVCRT:utility.obj
 0001:00002c18       __scrt_initialize_onexit_tables 0000000180003c18 f   MSVCRT:utility.obj
 0001:00002ca4       __scrt_is_nonwritable_in_current_image 0000000180003ca4 f   MSVCRT:utility.obj
 0001:00002d3c       __scrt_release_startup_lock 0000000180003d3c f   MSVCRT:utility.obj
 0001:00002d60       __scrt_uninitialize_crt    0000000180003d60 f   MSVCRT:utility.obj
 0001:00002d8c       _onexit                    0000000180003d8c f   MSVCRT:utility.obj
 0001:00002dc8       atexit                     0000000180003dc8 f   MSVCRT:utility.obj
 0001:00002de0       __crt_debugger_hook        0000000180003de0 f   MSVCRT:utility_desktop.obj
 0001:00002de8       __scrt_fastfail            0000000180003de8 f   MSVCRT:utility_desktop.obj
 0001:00002f34       _guard_check_icall_nop     0000000180003f34 f i MSVCRT:guard_support.obj
 0001:00002f38       __security_init_cookie     0000000180003f38 f   MSVCRT:gs_support.obj
 0001:00002fe4       DllMain                    0000000180003fe4 f   MSVCRT:dll_dllmain_stub.obj
 0001:00003008       ?__scrt_initialize_type_info@@YAXXZ 0000000180004008 f   MSVCRT:tncleanup.obj
 0001:00003018       ?__scrt_uninitialize_type_info@@YAXXZ 0000000180004018 f   MSVCRT:tncleanup.obj
 0001:00003024       __local_stdio_scanf_options 0000000180004024 f i MSVCRT:default_local_stdio_options.obj
 0001:0000302c       __scrt_initialize_default_local_stdio_options 000000018000402c f   MSVCRT:default_local_stdio_options.obj
 0001:00003048       __scrt_get_dyn_tls_init_callback 0000000180004048 f   MSVCRT:dyn_tls_init.obj
 0001:00003050       _RTC_Initialize            0000000180004050 f   MSVCRT:initsect.obj
 0001:0000308c       _RTC_Terminate             000000018000408c f   MSVCRT:initsect.obj
 0001:000030c8       __isa_available_init       00000001800040c8 f   MSVCRT:cpu_disp.obj
 0001:00003274       _get_startup_argv_mode     0000000180004274 f   MSVCRT:argv_mode.obj
 0001:0000327c       __scrt_is_ucrt_dll_in_use  000000018000427c f   MSVCRT:ucrt_detection.obj
 0001:00003290       memcpy                     0000000180004290 f   vcruntime:VCRUNTIME140.dll
 0001:00003296       memset                     0000000180004296 f   vcruntime:VCRUNTIME140.dll
 0001:0000329c       strchr                     000000018000429c f   vcruntime:VCRUNTIME140.dll
 0001:000032a2       __C_specific_handler       00000001800042a2 f   vcruntime:VCRUNTIME140.dll
 0001:000032a8       __std_type_info_destroy_list 00000001800042a8 f   vcruntime:VCRUNTIME140.dll
 0001:000032ae       strlen                     00000001800042ae f   ucrt:api-ms-win-crt-string-l1-1-0.dll
 0001:000032b4       _initterm                  00000001800042b4 f   ucrt:api-ms-win-crt-runtime-l1-1-0.dll
 0001:000032ba       _initterm_e                00000001800042ba f   ucrt:api-ms-win-crt-runtime-l1-1-0.dll
 0001:000032c0       _seh_filter_dll            00000001800042c0 f   ucrt:api-ms-win-crt-runtime-l1-1-0.dll
 0001:000032c6       _configure_narrow_argv     00000001800042c6 f   ucrt:api-ms-win-crt-runtime-l1-1-0.dll
 0001:000032cc       _initialize_narrow_environment 00000001800042cc f   ucrt:api-ms-win-crt-runtime-l1-1-0.dll
 0001:000032d2       _initialize_onexit_table   00000001800042d2 f   ucrt:api-ms-win-crt-runtime-l1-1-0.dll
 0001:000032d8       _register_onexit_function  00000001800042d8 f   ucrt:api-ms-win-crt-runtime-l1-1-0.dll
 0001:000032de       _execute_onexit_table      00000001800042de f   ucrt:api-ms-win-crt-runtime-l1-1-0.dll
 0001:000032e4       _crt_atexit                00000001800042e4 f   ucrt:api-ms-win-crt-runtime-l1-1-0.dll
 0001:000032ea       _cexit                     00000001800042ea f   ucrt:api-ms-win-crt-runtime-l1-1-0.dll
 0001:000032f0       __acrt_initialize          00000001800042f0 f   MSVCRT:ucrt_stubs.obj
 0001:000032f0       __acrt_thread_attach       00000001800042f0 f   MSVCRT:ucrt_stubs.obj
 0001:000032f0       __acrt_thread_detach       00000001800042f0 f   MSVCRT:ucrt_stubs.obj
 0001:000032f0       __acrt_uninitialize        00000001800042f0 f   MSVCRT:ucrt_stubs.obj
 0001:000032f0       __acrt_uninitialize_critical 00000001800042f0 f   MSVCRT:ucrt_stubs.obj
 0001:000032f0       __scrt_stub_for_acrt_initialize 00000001800042f0 f   MSVCRT:ucrt_stubs.obj
 0001:000032f0       __scrt_stub_for_acrt_thread_attach 00000001800042f0 f   MSVCRT:ucrt_stubs.obj
 0001:000032f0       __scrt_stub_for_acrt_thread_detach 00000001800042f0 f   MSVCRT:ucrt_stubs.obj
 0001:000032f0       __scrt_stub_for_acrt_uninitialize 00000001800042f0 f   MSVCRT:ucrt_stubs.obj
 0001:000032f0       __scrt_stub_for_acrt_uninitialize_critical 00000001800042f0 f   MSVCRT:ucrt_stubs.obj
 0001:000032f0       __vcrt_initialize          00000001800042f0 f   MSVCRT:ucrt_stubs.obj
 0001:000032f0       __vcrt_thread_attach       00000001800042f0 f   MSVCRT:ucrt_stubs.obj
 0001:000032f0       __vcrt_thread_detach       00000001800042f0 f   MSVCRT:ucrt_stubs.obj
 0001:000032f0       __vcrt_uninitialize        00000001800042f0 f   MSVCRT:ucrt_stubs.obj
 0001:000032f0       __vcrt_uninitialize_critical 00000001800042f0 f   MSVCRT:ucrt_stubs.obj
 0001:000032f4       __scrt_stub_for_is_c_termination_complete 00000001800042f4 f   MSVCRT:ucrt_stubs.obj
 0001:000032f4       _is_c_termination_complete 00000001800042f4 f   MSVCRT:ucrt_stubs.obj
 0001:00003310       _guard_dispatch_icall_nop  0000000180004310 f   MSVCRT:guard_dispatch.obj
 0001:00003330       _guard_xfg_dispatch_icall_nop 0000000180004330 f   MSVCRT:guard_xfg_dispatch.obj
 0002:00000000       __imp_RtlCaptureContext    0000000180005000     kernel32:KERNEL32.dll
 0002:00000008       __imp_RtlLookupFunctionEntry 0000000180005008     kernel32:KERNEL32.dll
 0002:00000010       __imp_RtlVirtualUnwind     0000000180005010     kernel32:KERNEL32.dll
 0002:00000018       __imp_UnhandledExceptionFilter 0000000180005018     kernel32:KERNEL32.dll
 0002:00000020       __imp_SetUnhandledExceptionFilter 0000000180005020     kernel32:KERNEL32.dll
 0002:00000028       __imp_GetCurrentProcess    0000000180005028     kernel32:KERNEL32.dll
 0002:00000030       __imp_TerminateProcess     0000000180005030     kernel32:KERNEL32.dll
 0002:00000038       __imp_IsProcessorFeaturePresent 0000000180005038     kernel32:KERNEL32.dll
 0002:00000040       __imp_CloseHandle          0000000180005040     kernel32:KERNEL32.dll
 0002:00000048       __imp_InitializeCriticalSectionAndSpinCount 0000000180005048     kernel32:KERNEL32.dll
 0002:00000050       __imp_DeleteCriticalSection 0000000180005050     kernel32:KERNEL32.dll
 0002:00000058       __imp_CreateEventW         0000000180005058     kernel32:KERNEL32.dll
 0002:00000060       __imp_GetModuleHandleW     0000000180005060     kernel32:KERNEL32.dll
 0002:00000068       __imp_GetProcAddress       0000000180005068     kernel32:KERNEL32.dll
 0002:00000070       __imp_IsDebuggerPresent    0000000180005070     kernel32:KERNEL32.dll
 0002:00000078       __imp_QueryPerformanceCounter 0000000180005078     kernel32:KERNEL32.dll
 0002:00000080       __imp_GetCurrentProcessId  0000000180005080     kernel32:KERNEL32.dll
 0002:00000088       __imp_GetCurrentThreadId   0000000180005088     kernel32:KERNEL32.dll
 0002:00000090       __imp_GetSystemTimeAsFileTime 0000000180005090     kernel32:KERNEL32.dll
 0002:00000098       __imp_DisableThreadLibraryCalls 0000000180005098     kernel32:KERNEL32.dll
 0002:000000a0       __imp_InitializeSListHead  00000001800050a0     kernel32:KERNEL32.dll
 0002:000000a8       \177KERNEL32_NULL_THUNK_DATA 00000001800050a8     kernel32:KERNEL32.dll
 0002:000000b0       __imp_memcpy               00000001800050b0     vcruntime:VCRUNTIME140.dll
 0002:000000b8       __imp_memset               00000001800050b8     vcruntime:VCRUNTIME140.dll
 0002:000000c0       __imp_strchr               00000001800050c0     vcruntime:VCRUNTIME140.dll
 0002:000000c8       __imp___C_specific_handler 00000001800050c8     vcruntime:VCRUNTIME140.dll
 0002:000000d0       __imp___std_type_info_destroy_list 00000001800050d0     vcruntime:VCRUNTIME140.dll
 0002:000000d8       \177VCRUNTIME140_NULL_THUNK_DATA 00000001800050d8     vcruntime:VCRUNTIME140.dll
 0002:000000e0       __imp_malloc               00000001800050e0     ucrt:api-ms-win-crt-heap-l1-1-0.dll
 0002:000000e8       __imp_free                 00000001800050e8     ucrt:api-ms-win-crt-heap-l1-1-0.dll
 0002:000000f0       \177api-ms-win-crt-heap-l1-1-0_NULL_THUNK_DATA 00000001800050f0     ucrt:api-ms-win-crt-heap-l1-1-0.dll
 0002:000000f8       __imp__errno               00000001800050f8     ucrt:api-ms-win-crt-runtime-l1-1-0.dll
 0002:00000100       __imp_exit                 0000000180005100     ucrt:api-ms-win-crt-runtime-l1-1-0.dll
 0002:00000108       __imp__cexit               0000000180005108     ucrt:api-ms-win-crt-runtime-l1-1-0.dll
 0002:00000110       __imp__crt_atexit          0000000180005110     ucrt:api-ms-win-crt-runtime-l1-1-0.dll
 0002:00000118       __imp__execute_onexit_table 0000000180005118     ucrt:api-ms-win-crt-runtime-l1-1-0.dll
 0002:00000120       __imp__register_onexit_function 0000000180005120     ucrt:api-ms-win-crt-runtime-l1-1-0.dll
 0002:00000128       __imp__initialize_onexit_table 0000000180005128     ucrt:api-ms-win-crt-runtime-l1-1-0.dll
 0002:00000130       __imp__initialize_narrow_environment 0000000180005130     ucrt:api-ms-win-crt-runtime-l1-1-0.dll
 0002:00000138       __imp__configure_narrow_argv 0000000180005138     ucrt:api-ms-win-crt-runtime-l1-1-0.dll
 0002:00000140       __imp__seh_filter_dll      0000000180005140     ucrt:api-ms-win-crt-runtime-l1-1-0.dll
 0002:00000148       __imp__initterm_e          0000000180005148     ucrt:api-ms-win-crt-runtime-l1-1-0.dll
 0002:00000150       __imp__initterm            0000000180005150     ucrt:api-ms-win-crt-runtime-l1-1-0.dll
 0002:00000158       \177api-ms-win-crt-runtime-l1-1-0_NULL_THUNK_DATA 0000000180005158     ucrt:api-ms-win-crt-runtime-l1-1-0.dll
 0002:00000160       __imp___acrt_iob_func      0000000180005160     ucrt:api-ms-win-crt-stdio-l1-1-0.dll
 0002:00000168       __imp_fflush               0000000180005168     ucrt:api-ms-win-crt-stdio-l1-1-0.dll
 0002:00000170       __imp___stdio_common_vsprintf 0000000180005170     ucrt:api-ms-win-crt-stdio-l1-1-0.dll
 0002:00000178       __imp___stdio_common_vfprintf 0000000180005178     ucrt:api-ms-win-crt-stdio-l1-1-0.dll
 0002:00000180       \177api-ms-win-crt-stdio-l1-1-0_NULL_THUNK_DATA 0000000180005180     ucrt:api-ms-win-crt-stdio-l1-1-0.dll
 0002:00000188       __imp__strdup              0000000180005188     ucrt:api-ms-win-crt-string-l1-1-0.dll
 0002:00000188       __imp_strdup               0000000180005188     ucrt:api-ms-win-crt-string-l1-1-0.dll
 0002:00000190       __imp_strlen               0000000180005190     ucrt:api-ms-win-crt-string-l1-1-0.dll
 0002:00000198       __imp_strncpy              0000000180005198     ucrt:api-ms-win-crt-string-l1-1-0.dll
 0002:000001a0       \177api-ms-win-crt-string-l1-1-0_NULL_THUNK_DATA 00000001800051a0     ucrt:api-ms-win-crt-string-l1-1-0.dll
 0002:000001a8       __guard_check_icall_fptr   00000001800051a8     MSVCRT:guard_support.obj
 0002:000001b0       __guard_xfg_check_icall_fptr 00000001800051b0     MSVCRT:guard_support.obj
 0002:000001b8       __guard_dispatch_icall_fptr 00000001800051b8     MSVCRT:guard_support.obj
 0002:000001c0       __guard_xfg_dispatch_icall_fptr 00000001800051c0     MSVCRT:guard_support.obj
 0002:000001c8       __guard_xfg_table_dispatch_icall_fptr 00000001800051c8     MSVCRT:guard_support.obj
 0002:000001d0       __castguard_check_failure_os_handled_fptr 00000001800051d0     MSVCRT:guard_support.obj
 0002:000001d8       __guard_memcpy_fptr        00000001800051d8     vcruntime:softmemtag.obj
 0002:000001e0       __xc_a                     00000001800051e0     MSVCRT:initializers.obj
 0002:000001e8       __xc_z                     00000001800051e8     MSVCRT:initializers.obj
 0002:000001f0       __xi_a                     00000001800051f0     MSVCRT:initializers.obj
 0002:00000200       __xi_z                     0000000180005200     MSVCRT:initializers.obj
 0002:00000208       __xl_a                     0000000180005208     MSVCRT:tlssup.obj
 0002:00000210       __xl_z                     0000000180005210     MSVCRT:tlssup.obj
 0002:00000218       __xp_a                     0000000180005218     MSVCRT:initializers.obj
 0002:00000220       __xp_z                     0000000180005220     MSVCRT:initializers.obj
 0002:00000228       __xt_a                     0000000180005228     MSVCRT:initializers.obj
 0002:00000230       __xt_z                     0000000180005230     MSVCRT:initializers.obj
 0002:00000240       g_refKindStr               0000000180005240     libHeap.obj
 0002:000003f0       ??_C@_09BPLDFGCI@unknown_0@ 00000001800053f0     libHeap.obj
 0002:00000400       ??_C@_0BL@FPNMECJD@JVMTI_HEAP_REFERENCE_CLASS@ 0000000180005400     libHeap.obj
 0002:00000420       ??_C@_0BL@FKGKKLNM@JVMTI_HEAP_REFERENCE_FIELD@ 0000000180005420     libHeap.obj
 0002:00000440       ??_C@_0CD@CAEHCFJF@JVMTI_HEAP_REFERENCE_ARRAY_ELEM@ 0000000180005440     libHeap.obj
 0002:00000468       ??_C@_0CC@DNEBMCNK@JVMTI_HEAP_REFERENCE_CLASS_LOAD@ 0000000180005468     libHeap.obj
 0002:00000490       ??_C@_0BN@CJMIPEBB@JVMTI_HEAP_REFERENCE_SIGNERS@ 0000000180005490     libHeap.obj
 0002:000004b0       ??_C@_0CH@HBOIDPEB@JVMTI_HEAP_REFERENCE_PROTECTION@ 00000001800054b0     libHeap.obj
 0002:000004d8       ??_C@_0BP@MDKGDGKL@JVMTI_HEAP_REFERENCE_INTERFACE@ 00000001800054d8     libHeap.obj
 0002:000004f8       ??_C@_0CC@JJMIHNJH@JVMTI_HEAP_REFERENCE_STATIC_FIE@ 00000001800054f8     libHeap.obj
 0002:00000520       ??_C@_0CD@IDHEEGID@JVMTI_HEAP_REFERENCE_CONSTANT_P@ 0000000180005520     libHeap.obj
 0002:00000548       ??_C@_0CA@EFFCHNG@JVMTI_HEAP_REFERENCE_SUPERCLASS@ 0000000180005548     libHeap.obj
 0002:00000568       ??_C@_0L@PCDFHGCJ@unknown_11@ 0000000180005568     libHeap.obj
 0002:00000578       ??_C@_0L@NJBICFOK@unknown_12@ 0000000180005578     libHeap.obj
 0002:00000588       ??_C@_0L@MAADBEKL@unknown_13@ 0000000180005588     libHeap.obj
 0002:00000598       ??_C@_0L@IPECICGM@unknown_14@ 0000000180005598     libHeap.obj
 0002:000005a8       ??_C@_0L@JGFJLDCN@unknown_15@ 00000001800055a8     libHeap.obj
 0002:000005b8       ??_C@_0L@LNHEOAOO@unknown_16@ 00000001800055b8     libHeap.obj
 0002:000005c8       ??_C@_0L@KEGPNBKP@unknown_17@ 00000001800055c8     libHeap.obj
 0002:000005d8       ??_C@_0L@CDPHMNGA@unknown_18@ 00000001800055d8     libHeap.obj
 0002:000005e8       ??_C@_0L@DKOMPMCB@unknown_19@ 00000001800055e8     libHeap.obj
 0002:000005f8       ??_C@_0L@OJGIPJDB@unknown_20@ 00000001800055f8     libHeap.obj
 0002:00000608       ??_C@_0CA@KAOFNDEM@JVMTI_HEAP_REFERENCE_JNI_GLOBAL@ 0000000180005608     libHeap.obj
 0002:00000628       ??_C@_0CC@HPFAJBK@JVMTI_HEAP_REFERENCE_SYSTEM_CLA@ 0000000180005628     libHeap.obj
 0002:00000650       ??_C@_0BN@FDEGFOHC@JVMTI_HEAP_REFERENCE_MONITOR@ 0000000180005650     libHeap.obj
 0002:00000670       ??_C@_0CB@HKIBCMAJ@JVMTI_HEAP_REFERENCE_STACK_LOCA@ 0000000180005670     libHeap.obj
 0002:00000698       ??_C@_0BP@EAACMMOE@JVMTI_HEAP_REFERENCE_JNI_LOCAL@ 0000000180005698     libHeap.obj
 0002:000006b8       ??_C@_0BM@IJDEOGOE@JVMTI_HEAP_REFERENCE_THREAD@ 00000001800056b8     libHeap.obj
 0002:000006d8       ??_C@_0BL@EDGPPKC@JVMTI_HEAP_REFERENCE_OTHER@ 00000001800056d8     libHeap.obj
 0002:000006f4       ??_C@_04BCJPDBDA@Code@     00000001800056f4     libHeap.obj
 0002:00000700       ??_C@_0BA@OCLMCFKC@LineNumberTable@ 0000000180005700     libHeap.obj
 0002:00000710       ??_C@_0BD@CPAEPILC@LocalVariableTable@ 0000000180005710     libHeap.obj
 0002:00000728       ??_C@_0BH@NMBDNHBD@LocalVariableTypeTable@ 0000000180005728     libHeap.obj
 0002:00000740       ??_C@_0O@HIHEEDNJ@StackMapTable@ 0000000180005740     libHeap.obj
 0002:00000750       ??_C@_0L@HCDIAMJG@?9?5?$CFs?0?5?$CFd?3?5@ 0000000180005750     libHeap.obj
 0002:00000760       ??_C@_0JI@HLPECLFI@?$CD?5?4?4?4?6?$CD?5ERROR?3?5too?5many?5complai@ 0000000180005760     libHeap.obj
 0002:00000800       ??_C@_0ED@JNEKCCOB@The?5following?5fake?5exception?5st@ 0000000180005800     libHeap.obj
 0002:00000848       ??_C@_0CN@FCNMDFBH@nsk?4share?4Fake_Exception_for_RU@ 0000000180005848     libHeap.obj
 0002:00000878       ??_C@_08PGFFNAEI@?$CI?$CFs?3?$CFd?$CJ?5@ 0000000180005878     libHeap.obj
 0002:00000888       ??_C@_0DP@IENMAEGI@s?2test?2hotspot?2jtreg?2vmTestbase@ 0000000180005888     libHeap.obj
 0002:000008c8       ??_C@_0BL@NDJLFFJB@?7at?5nsk_lvcomplain?$CI?$CFs?3?$CFd?$CJ?6@ 00000001800058c8     libHeap.obj
 0002:000008e8       ??_C@_0BC@JOOKAFKF@?$CD?5ERROR?3?5?$CFs?0?5?$CFd?3?5@ 00000001800058e8     libHeap.obj
 0002:00000900       ??_C@_09KJEAHMEH@?$CD?5ERROR?3?5@ 0000000180005900     libHeap.obj
 0002:0000090c       ??_C@_02GPIOPFAK@?$DO?$DO@ 000000018000590c     libHeap.obj
 0002:00000910       ??_C@_02FODMEDOG@?$DM?$DM@ 0000000180005910     libHeap.obj
 0002:00000914       ??_C@_02DJGKEECL@?4?4@     0000000180005914     libHeap.obj
 0002:00000918       ??_C@_0O@CJPGJOAF@?9?5?$CFs?0?5?$CFd?3?5?$CFs?5@ 0000000180005918     libHeap.obj
 0002:00000928       ??_C@_0CB@IAKPDOIC@?$CD?5?5?5verified?5assertion?5is?5FALSE@ 0000000180005928     libHeap.obj
 0002:00000950       ??_C@_0CO@LGONDEPD@stdout?3?5fflush?5failed?5?9?5err?$DN?$CFd?5@ 0000000180005950     libHeap.obj
 0002:00000980       ??_C@_0CO@KBGKJPBD@stderr?3?5fflush?5failed?5?9?5err?$DN?$CFd?5@ 0000000180005980     libHeap.obj
 0002:000009b0       ??_C@_0BB@JCNMKLLK@JVMTI_ERROR_NONE@ 00000001800059b0     libHeap.obj
 0002:000009c8       ??_C@_0BL@LDIMKLPH@JVMTI_ERROR_INVALID_THREAD@ 00000001800059c8     libHeap.obj
 0002:000009e8       ??_C@_0CB@PJFPAIKJ@JVMTI_ERROR_INVALID_THREAD_GROU@ 00000001800059e8     libHeap.obj
 0002:00000a10       ??_C@_0BN@LLMKHMNF@JVMTI_ERROR_INVALID_PRIORITY@ 0000000180005a10     libHeap.obj
 0002:00000a30       ??_C@_0CB@MBOFKAGB@JVMTI_ERROR_THREAD_NOT_SUSPENDE@ 0000000180005a30     libHeap.obj
 0002:00000a58       ??_C@_0BN@FABOLPBI@JVMTI_ERROR_THREAD_SUSPENDED@ 0000000180005a58     libHeap.obj
 0002:00000a78       ??_C@_0BN@FDGNOBJM@JVMTI_ERROR_THREAD_NOT_ALIVE@ 0000000180005a78     libHeap.obj
 0002:00000a98       ??_C@_0BL@GOBIFKNJ@JVMTI_ERROR_INVALID_OBJECT@ 0000000180005a98     libHeap.obj
 0002:00000ab8       ??_C@_0BK@FCMAJPPC@JVMTI_ERROR_INVALID_CLASS@ 0000000180005ab8     libHeap.obj
 0002:00000ad8       ??_C@_0BP@IKLLBKEB@JVMTI_ERROR_CLASS_NOT_PREPARED@ 0000000180005ad8     libHeap.obj
 0002:00000af8       ??_C@_0BN@KLPPLKG@JVMTI_ERROR_INVALID_METHODID@ 0000000180005af8     libHeap.obj
 0002:00000b18       ??_C@_0BN@BCEKOKND@JVMTI_ERROR_INVALID_LOCATION@ 0000000180005b18     libHeap.obj
 0002:00000b38       ??_C@_0BM@DFDGPME@JVMTI_ERROR_INVALID_FIELDID@ 0000000180005b38     libHeap.obj
 0002:00000b58       ??_C@_0BL@NELIEPEC@JVMTI_ERROR_NO_MORE_FRAMES@ 0000000180005b58     libHeap.obj
 0002:00000b78       ??_C@_0BJ@BDBECFDM@JVMTI_ERROR_OPAQUE_FRAME@ 0000000180005b78     libHeap.obj
 0002:00000b98       ??_C@_0BK@MIIFNLOB@JVMTI_ERROR_TYPE_MISMATCH@ 0000000180005b98     libHeap.obj
 0002:00000bb8       ??_C@_0BJ@HPCAOILC@JVMTI_ERROR_INVALID_SLOT@ 0000000180005bb8     libHeap.obj
 0002:00000bd8       ??_C@_0BG@CHILOPNI@JVMTI_ERROR_DUPLICATE@ 0000000180005bd8     libHeap.obj
 0002:00000bf0       ??_C@_0BG@DIEMLHKM@JVMTI_ERROR_NOT_FOUND@ 0000000180005bf0     libHeap.obj
 0002:00000c08       ??_C@_0BM@NHMCKHOB@JVMTI_ERROR_INVALID_MONITOR@ 0000000180005c08     libHeap.obj
 0002:00000c28       ??_C@_0BO@PPEDAJGL@JVMTI_ERROR_NOT_MONITOR_OWNER@ 0000000180005c28     libHeap.obj
 0002:00000c48       ??_C@_0BG@FCAIPEID@JVMTI_ERROR_INTERRUPT@ 0000000180005c48     libHeap.obj
 0002:00000c60       ??_C@_0CB@EGDBNKOI@JVMTI_ERROR_INVALID_CLASS_FORMA@ 0000000180005c60     libHeap.obj
 0002:00000c88       ??_C@_0CG@DGKOGIAL@JVMTI_ERROR_CIRCULAR_CLASS_DEFI@ 0000000180005c88     libHeap.obj
 0002:00000cb0       ??_C@_0BP@ICEALPKC@JVMTI_ERROR_FAILS_VERIFICATION@ 0000000180005cb0     libHeap.obj
 0002:00000cd0       ??_C@_0DC@JDACLMIO@JVMTI_ERROR_UNSUPPORTED_REDEFIN@ 0000000180005cd0     libHeap.obj
 0002:00000d08       ??_C@_0DE@GKDKNOMJ@JVMTI_ERROR_UNSUPPORTED_REDEFIN@ 0000000180005d08     libHeap.obj
 0002:00000d40       ??_C@_0BO@LAFKIOG@JVMTI_ERROR_INVALID_TYPESTATE@ 0000000180005d40     libHeap.obj
 0002:00000d60       ??_C@_0DH@INDGCLLB@JVMTI_ERROR_UNSUPPORTED_REDEFIN@ 0000000180005d60     libHeap.obj
 0002:00000d98       ??_C@_0DE@NHEOMMGI@JVMTI_ERROR_UNSUPPORTED_REDEFIN@ 0000000180005d98     libHeap.obj
 0002:00000dd0       ??_C@_0CA@EKPNJOEP@JVMTI_ERROR_UNSUPPORTED_VERSION@ 0000000180005dd0     libHeap.obj
 0002:00000df0       ??_C@_0BN@OFFMAHHL@JVMTI_ERROR_NAMES_DONT_MATCH@ 0000000180005df0     libHeap.obj
 0002:00000e10       ??_C@_0DN@HHBBLAKE@JVMTI_ERROR_UNSUPPORTED_REDEFIN@ 0000000180005e10     libHeap.obj
 0002:00000e50       ??_C@_0DO@HMBGBGNA@JVMTI_ERROR_UNSUPPORTED_REDEFIN@ 0000000180005e50     libHeap.obj
 0002:00000e90       ??_C@_0BP@PBECGKHJ@JVMTI_ERROR_UNMODIFIABLE_CLASS@ 0000000180005e90     libHeap.obj
 0002:00000eb0       ??_C@_0BK@CANILEHF@JVMTI_ERROR_NOT_AVAILABLE@ 0000000180005eb0     libHeap.obj
 0002:00000ed0       ??_C@_0CE@INJKMEFK@JVMTI_ERROR_MUST_POSSESS_CAPABI@ 0000000180005ed0     libHeap.obj
 0002:00000ef8       ??_C@_0BJ@LBFPFPDM@JVMTI_ERROR_NULL_POINTER@ 0000000180005ef8     libHeap.obj
 0002:00000f18       ??_C@_0BP@CHJPNNEM@JVMTI_ERROR_ABSENT_INFORMATION@ 0000000180005f18     libHeap.obj
 0002:00000f38       ??_C@_0BP@OMFMNLC@JVMTI_ERROR_INVALID_EVENT_TYPE@ 0000000180005f38     libHeap.obj
 0002:00000f58       ??_C@_0BN@BIBNPHHO@JVMTI_ERROR_ILLEGAL_ARGUMENT@ 0000000180005f58     libHeap.obj
 0002:00000f78       ??_C@_0BK@KKNDHDCE@JVMTI_ERROR_NATIVE_METHOD@ 0000000180005f78     libHeap.obj
 0002:00000f98       ??_C@_0BK@PMKCFHAE@JVMTI_ERROR_OUT_OF_MEMORY@ 0000000180005f98     libHeap.obj
 0002:00000fb8       ??_C@_0BK@NNJBDMNB@JVMTI_ERROR_ACCESS_DENIED@ 0000000180005fb8     libHeap.obj
 0002:00000fd8       ??_C@_0BI@GHECLMNC@JVMTI_ERROR_WRONG_PHASE@ 0000000180005fd8     libHeap.obj
 0002:00000ff0       ??_C@_0BF@OLIHJOII@JVMTI_ERROR_INTERNAL@ 0000000180005ff0     libHeap.obj
 0002:00001008       ??_C@_0BO@EOHGKJHI@JVMTI_ERROR_UNATTACHED_THREAD@ 0000000180006008     libHeap.obj
 0002:00001028       ??_C@_0CA@LKHFDACL@JVMTI_ERROR_INVALID_ENVIRONMENT@ 0000000180006028     libHeap.obj
 0002:00001048       ??_C@_0BA@MMFHLOKK@?$DMunknown?5error?$DO@ 0000000180006048     libHeap.obj
 0002:00001058       ??_C@_0CF@CBHOKDB@throwable?5?$DN?5jni?9?$DOExceptionOccur@ 0000000180006058     libHeap.obj
 0002:00001080       ??_C@_03OFAPEBGM@?$CFs?6@  0000000180006080     libHeap.obj
 0002:00001088       ??_C@_0DM@LPIGEGNJ@s?2test?2hotspot?2jtreg?2vmTestbase@ 0000000180006088     libHeap.obj
 0002:000010c8       ??_C@_0CC@NFCNPEPK@Exception?5in?5JNI?5call?5?$CIcleared?$CJ@ 00000001800060c8     libHeap.obj
 0002:000010f0       ??_C@_0BJ@IBAKFIKF@jni?9?$DOExceptionDescribe?$CI?$CJ@ 00000001800060f0     libHeap.obj
 0002:00001110       ??_C@_0BG@GGKALKMH@jni?9?$DOExceptionClear?$CI?$CJ@ 0000000180006110     libHeap.obj
 0002:00001128       ??_C@_0CF@JMGFGJLJ@?$CD?5?5?5verified?5JNI?5assertion?5is?5F@ 0000000180006128     libHeap.obj
 0002:00001150       ??_C@_0CB@MLNJNCLJ@?5?5jvmti?5error?3?5code?$DN?$CFd?0?5name?$DN?$CFs@ 0000000180006150     libHeap.obj
 0002:00001178       ??_C@_0CD@OHBGDKMK@?$CD?5?5?5jvmti?5error?3?5code?$DN?$CFd?0?5name?$DN@ 0000000180006178     libHeap.obj
 0002:000011a0       ??_C@_0CG@JNNCGPHB@?$CD?5?5?5error?5expected?3?5code?$DN?$CFd?0?5na@ 00000001800061a0     libHeap.obj
 0002:000011d0       ??_C@_0EB@IMGKPCGE@?$CIstr_obj?5?$DN?5jni?9?$DONewStringUTF?$CIco@ 00000001800061d0     libHeap.obj
 0002:00001220       ??_C@_0EA@HFOGGBCC@s?2test?2hotspot?2jtreg?2vmTestbase@ 0000000180006220     libHeap.obj
 0002:00001260       ??_C@_05KKCIMGE@error@     0000000180006260     libHeap.obj
 0002:00001268       ??_C@_0CJ@JACLEAA@Test?5failed?5by?5setFailStatus?$CI?$CJ?4@ 0000000180006268     libHeap.obj
 0002:000012a0       ??_C@_0EA@PNBCDMOA@s?2test?2hotspot?2jtreg?2vmTestbase@ 00000001800062a0     libHeap.obj
 0002:000012e0       ??_C@_0DI@ILAHDLMP@?$CI?$CKagentThreadProc?$CJ?$CIjvmti_env?0?5a@ 00000001800062e0     libHeap.obj
 0002:00001318       ??_C@_0BD@KDBALNLB@JVMTI?5agent?5thread@ 0000000180006318     libHeap.obj
 0002:00001330       ??_C@_0BB@NOKBFPFO@java?1lang?1Thread@ 0000000180006330     libHeap.obj
 0002:00001344       ??_C@_06FALKBLGB@?$DMinit?$DO@ 0000000180006344     libHeap.obj
 0002:00001350       ??_C@_0BG@IKDDPPGD@?$CILjava?1lang?1String?$DL?$CJV@ 0000000180006350     libHeap.obj
 0002:00001370       ??_C@_0EB@IFJBFEKC@?$CIthreadClass?5?$DN?5jni_env?9?$DOFindCla@ 0000000180006370     libHeap.obj
 0002:000013c0       ??_C@_0GF@FGFIBKKL@?$CIthreadCtor?5?$DN?5jni_env?9?$DOGetMetho@ 00000001800063c0     libHeap.obj
 0002:00001428       ??_C@_0DN@NCPDJLOG@?$CIthreadName?5?$DN?5jni_env?9?$DONewStrin@ 0000000180006428     libHeap.obj
 0002:00001470       ??_C@_0FE@PFKODBGC@?$CIthreadObject?5?$DN?5jni_env?9?$DONewObj@ 0000000180006470     libHeap.obj
 0002:000014d0       ??_C@_0ED@HOBAHHJI@?$CIthreadGlobalRef?5?$DN?5jni_env?9?$DONew@ 00000001800064d0     libHeap.obj
 0002:00001520       ??_C@_0FN@HNJJAHFC@jvmti_env?9?$DORunAgentThread?$CIagent@ 0000000180006520     libHeap.obj
 0002:00001580       ??_C@_0EA@MOJDNKDF@Debuggee?5status?5sync?5aborted?5be@ 0000000180006580     libHeap.obj
 0002:000015c0       ??_C@_0EA@EEOEJAEN@status?5?$DN?5syncDebuggeeStatus?$CIjni@ 00000001800065c0     libHeap.obj
 0002:00001600       ??_C@_0BL@JBCFNBMB@nsk_jvmti_resetAgentData?$CI?$CJ@ 0000000180006600     libHeap.obj
 0002:00001620       ??_C@_0EL@LPBEELIP@s?2test?2hotspot?2jtreg?2vmTestbase@ 0000000180006620     libHeap.obj
 0002:00001670       ??_C@_0CK@JDAMFDMJ@jvmti?9?$DOSetTag?$CIo?0?5tag?$CJ?5?$DN?$DN?5JVMTI_@ 0000000180006670     libHeap.obj
 0002:000016a0       ??_C@_0CC@DAMNHKNI@Can?8t?5set?5tag?5?$CFli?5for?5object?5?$CFl@ 00000001800066a0     libHeap.obj
 0002:000016c8       ??_C@_0DL@HAJPNKEF@jvmti?9?$DOGetObjectHashCode?$CIo?0?5?$CGha@ 00000001800066c8     libHeap.obj
 0002:00001708       ??_C@_0BL@JFPIEOBF@Can?8t?5get?5hash?5object?5?$CFlx?6@ 0000000180006708     libHeap.obj
 0002:00001728       ??_C@_0BG@DICPHBKN@setTag?3?5?$CF08x?5?$DM?9?5?$CF?53li@ 0000000180006728     libHeap.obj
 0002:00001740       ??_C@_0DH@FCEEBDMJ@?$CIs?5?$DN?5jni?9?$DOGetStringUTFChars?$CIsIn@ 0000000180006740     libHeap.obj
 0002:00001778       ??_C@_0BJ@OKKGHDCN@Can?8t?5get?5string?5at?5?$CF?$CDp?6@ 0000000180006778     libHeap.obj
 0002:00001798       ??_C@_0BP@EKFLGGFJ@Can?8t?5get?5string?5at?5?$CF?$CDp?3?5null?6@ 0000000180006798     libHeap.obj
 0002:000017b8       ??_C@_06ICODBHCL@?5?1?1?5?$CFs@ 00000001800067b8     libHeap.obj
 0002:000017c0       ??_C@_0DB@KGFPLEGO@?$CIr?5?$DN?5jvmti?9?$DOGetTag?$CIo?0?5?$CGtag?$CJ?$CJ?5?$DN?$DN@ 00000001800067c0     libHeap.obj
 0002:000017f8       ??_C@_0CO@PDAGBCGJ@Can?8t?5GetTag?5for?5object?5?$CFlx?4?5Re@ 00000001800067f8     libHeap.obj
 0002:00001828       ??_C@_0CH@HPEODOHC@TEST_BUG?3?5Max?4?5number?5of?5refs?5r@ 0000000180006828     libHeap.obj
 0002:00001850       ??_C@_0DI@PHFCABIM@?$CIr?5?$DN?5jvmti?9?$DOGetTag?$CIfrom?0?5?$CGtagFr@ 0000000180006850     libHeap.obj
 0002:00001888       ??_C@_0DI@MDEGFNKD@TEST_BUG?3?5Can?8t?5GetTag?5for?5obje@ 0000000180006888     libHeap.obj
 0002:000018c0       ??_C@_0DE@MLELJAHM@?$CIr?5?$DN?5jvmti?9?$DOGetTag?$CIto?0?5?$CGtagTo?$CJ?$CJ@ 00000001800068c0     libHeap.obj
 0002:000018f8       ??_C@_0DC@EKMDGEGF@WARNING?3?5?$CIdefault?$CJ?5unexpected?5v@ 00000001800068f8     libHeap.obj
 0002:00001930       ??_C@_0CG@IAFCDBJK@ERORR?3?5GetTag?5failed?3?5JVMTI?5err@ 0000000180006930     libHeap.obj
 0002:00001958       ??_C@_0CN@CJLEGEAD@ERORR?3?5GetObjectSize?5failed?3?5JV@ 0000000180006958     libHeap.obj
 0002:00001988       ??_C@_0CL@NHCPFNKG@WARNING?3?5default?5heap_object_ca@ 0000000180006988     libHeap.obj
 0002:000019b8       ??_C@_0DD@IPHEJNH@IterateOverReachableObjects?5fai@ 00000001800069b8     libHeap.obj
 0002:000019f0       ??_C@_0DN@JAKBPEFB@IterateOverObjectsReachableFrom@ 00000001800069f0     libHeap.obj
 0002:00001a30       ??_C@_0CG@CKGGGLA@ERROR?3?5GetObjectsWithTags?5faile@ 0000000180006a30     libHeap.obj
 0002:00001a58       ??_C@_0BB@DDFKOHA@java?1lang?1Object@ 0000000180006a58     libHeap.obj
 0002:00001a70       ??_C@_0DB@FMNJGLJD@WARNING?3?5?$CItagged?$CJ?5unexpected?5va@ 0000000180006a70     libHeap.obj
 0002:00001aa8       ??_C@_0DA@JIIOMMFC@WARNING?3?5?$CItotal?$CJ?5unexpected?5val@ 0000000180006aa8     libHeap.obj
 0002:00001ad8       ??_C@_0DA@LEOIKFPB@WARNING?3?5?$CIklass?$CJ?5unexpected?5val@ 0000000180006ad8     libHeap.obj
 0002:00001b08       ??_C@_0CP@GAEGKLFH@WARNING?3?5?$CIheap?$CJ?5unexpected?5valu@ 0000000180006b08     libHeap.obj
 0002:00001b38       ??_C@_0CM@NLAMPGNM@WARNING?3?5jmethodID?5missing?5for?5@ 0000000180006b38     libHeap.obj
 0002:00001b68       ??_C@_0DA@JNIOIPNA@WARNING?3?5?$CIstack?$CJ?5unexpected?5val@ 0000000180006b68     libHeap.obj
 0002:00001b98       ??_C@_0DB@MCDDKPPH@WARNING?3?5?$CIobject?$CJ?5unexpected?5va@ 0000000180006b98     libHeap.obj
 0002:00001bd0       ??_C@_0DB@GBANCAIP@WARNING?3?5OBJECT_FREE?5event?5call@ 0000000180006bd0     libHeap.obj
 0002:00001c08       ??_C@_0DE@DGONBEPN@Unable?5to?5create?5jvmtiEnv?0?5GetE@ 0000000180006c08     libHeap.obj
 0002:00001c40       ??_C@_0CC@MOMJJHKJ@GetCapabilities?5failed?0?5error?$DN?$CF@ 0000000180006c40     libHeap.obj
 0002:00001c68       ??_C@_0CC@DOGPIPAH@AddCapabilities?5failed?0?5error?$DN?$CF@ 0000000180006c68     libHeap.obj
 0002:00001c90       ??_C@_0CL@IODBIPJN@SetEventNotificationMode?5failed@ 0000000180006c90     libHeap.obj
 0002:00001cc0       ??_C@_0CE@NIODJPMK@SetEventCallbacks?5failed?0?5error@ 0000000180006cc0     libHeap.obj
 0002:00001d00       ??_C@_1EC@JIJBPKFM@?$AAa?$AAp?$AAi?$AA?9?$AAm?$AAs?$AA?9?$AAw?$AAi?$AAn?$AA?9?$AAc?$AAo?$AAr?$AAe@ 0000000180006d00     MSVCRT:thread_safe_statics.obj
 0002:00001d48       ??_C@_1BK@MGMFAEKH@?$AAk?$AAe?$AAr?$AAn?$AAe?$AAl?$AA3?$AA2?$AA?4?$AAd?$AAl?$AAl@ 0000000180006d48     MSVCRT:thread_safe_statics.obj
 0002:00001d68       ??_C@_0BJ@JEBJOJFJ@SleepConditionVariableCS@ 0000000180006d68     MSVCRT:thread_safe_statics.obj
 0002:00001d88       ??_C@_0BJ@PGPPEPCC@WakeAllConditionVariable@ 0000000180006d88     MSVCRT:thread_safe_statics.obj
 0002:00001da8       _pDefaultRawDllMain        0000000180006da8     MSVCRT:dll_dllmain.obj
 0002:00001da8       _pRawDllMain               0000000180006da8     MSVCRT:dll_dllmain.obj
 0002:00001db0       __xmm@ffffffffffffffffffffffffffffffff 0000000180006db0     MSVCRT:utility.obj
 0002:00001dc0       _load_config_used          0000000180006dc0     MSVCRT:loadcfg.obj
 0002:00001f80       _tls_used                  0000000180006f80     MSVCRT:tlssup.obj
 0002:00001fa8       __volatile_metadata        0000000180006fa8     <linker-defined>
 0002:00002360       __rtc_iaa                  0000000180007360     MSVCRT:initsect.obj
 0002:00002368       __rtc_izz                  0000000180007368     MSVCRT:initsect.obj
 0002:00002370       __rtc_taa                  0000000180007370     MSVCRT:initsect.obj
 0002:00002378       __rtc_tzz                  0000000180007378     MSVCRT:initsect.obj
 0002:00002380       _tls_start                 0000000180007380     MSVCRT:tlssup.obj
 0002:00002384       _Init_thread_epoch         0000000180007384     MSVCRT:thread_safe_statics.obj
 0002:00002388       _tls_end                   0000000180007388     MSVCRT:tlssup.obj
 0002:00002f38       __IMPORT_DESCRIPTOR_KERNEL32 0000000180007f38     kernel32:KERNEL32.dll
 0002:00002f4c       __IMPORT_DESCRIPTOR_VCRUNTIME140 0000000180007f4c     vcruntime:VCRUNTIME140.dll
 0002:00002f60       __IMPORT_DESCRIPTOR_api-ms-win-crt-heap-l1-1-0 0000000180007f60     ucrt:api-ms-win-crt-heap-l1-1-0.dll
 0002:00002f74       __IMPORT_DESCRIPTOR_api-ms-win-crt-runtime-l1-1-0 0000000180007f74     ucrt:api-ms-win-crt-runtime-l1-1-0.dll
 0002:00002f88       __IMPORT_DESCRIPTOR_api-ms-win-crt-stdio-l1-1-0 0000000180007f88     ucrt:api-ms-win-crt-stdio-l1-1-0.dll
 0002:00002f9c       __IMPORT_DESCRIPTOR_api-ms-win-crt-string-l1-1-0 0000000180007f9c     ucrt:api-ms-win-crt-string-l1-1-0.dll
 0002:00002fb0       __NULL_IMPORT_DESCRIPTOR   0000000180007fb0     kernel32:KERNEL32.dll
 0003:00000038       _Init_global_epoch         0000000180009038     MSVCRT:thread_safe_statics.obj
 0003:00000040       __security_cookie          0000000180009040     MSVCRT:gs_cookie.obj
 0003:00000048       __security_cookie_complement 0000000180009048     MSVCRT:gs_cookie.obj
 0003:00000050       __scrt_native_dllmain_reason 0000000180009050     MSVCRT:utility.obj
 0003:00000058       __isa_available            0000000180009058     MSVCRT:cpu_disp.obj
 0003:0000005c       __isa_enabled              000000018000905c     MSVCRT:cpu_disp.obj
 0003:00000060       __memset_fast_string_threshold 0000000180009060     MSVCRT:cpu_disp.obj
 0003:00000068       __memset_nt_threshold      0000000180009068     MSVCRT:cpu_disp.obj
 0003:00000070       __scrt_ucrt_dll_is_in_use  0000000180009070     MSVCRT:ucrt_stubs.obj
 0003:00000080       g_wrongHeapCallbacks       0000000180009080     libHeap.obj
 0003:00000100       g_szTagInfo                0000000180009100     libHeap.obj
 0003:00002040       g_tagFlags                 000000018000b040     libHeap.obj
 0003:00002428       g_refsToVerifyCnt          000000018000b428     libHeap.obj
 0003:0000242c       g_fakeUserData             000000018000b42c     libHeap.obj
 0003:00002430       g_tagVisitCount            000000018000b430     libHeap.obj
 0003:000033d0       g_refsToVerify             000000018000c3d0     libHeap.obj
 0003:0001aad0       g_userDataError            0000000180023ad0     libHeap.obj
 0003:0001aca8       ?_OptionsStorage@?1??__local_stdio_printf_options@@9@4_KA 0000000180023ca8     libHeap.obj
 0003:0001b268       _tls_index                 0000000180024268     MSVCRT:tlssup.obj
 0003:0001b270       __scrt_current_native_startup_state 0000000180024270     MSVCRT:utility.obj
 0003:0001b278       __scrt_native_startup_lock 0000000180024278     MSVCRT:utility.obj
 0003:0001b2b8       __scrt_debugger_hook_flag  00000001800242b8     MSVCRT:utility_desktop.obj
 0003:0001b2c0       ?__type_info_root_node@@3U__type_info_node@@A 00000001800242c0     MSVCRT:tncleanup.obj
 0003:0001b2d0       ?_OptionsStorage@?1??__local_stdio_scanf_options@@9@4_KA 00000001800242d0     MSVCRT:default_local_stdio_options.obj
 0003:0001b2d8       __favor                    00000001800242d8     MSVCRT:cpu_disp.obj
 0003:0001b2e0       __dyn_tls_init_callback    00000001800242e0     <common>

 entry point at        0001:00002a20

 Static symbols

 0000:fffd9000       .debug$S                   0000000180000000     Heap.exp
 0000:fffd9000       .debug$S                   0000000180000000     vcruntime:VCRUNTIME140.dll
 0000:fffd9000       .debug$S                   0000000180000000     vcruntime:VCRUNTIME140.dll
 0000:fffd9000       .debug$S                   0000000180000000     vcruntime:VCRUNTIME140.dll
 0000:fffd9000       .debug$S                   0000000180000000     vcruntime:VCRUNTIME140.dll
 0000:fffd9000       .debug$S                   0000000180000000     vcruntime:VCRUNTIME140.dll
 0000:fffd9000       .debug$S                   0000000180000000     vcruntime:VCRUNTIME140.dll
 0000:fffd9000       .debug$S                   0000000180000000     vcruntime:VCRUNTIME140.dll
 0000:fffd9000       .debug$S                   0000000180000000     ucrt:api-ms-win-crt-convert-l1-1-0.dll
 0002:ffffb000       .idata$6                   0000000180000000     ucrt:api-ms-win-crt-convert-l1-1-0.dll
 0000:fffd9000       .debug$S                   0000000180000000     ucrt:api-ms-win-crt-heap-l1-1-0.dll
 0000:fffd9000       .debug$S                   0000000180000000     ucrt:api-ms-win-crt-heap-l1-1-0.dll
 0000:fffd9000       .debug$S                   0000000180000000     ucrt:api-ms-win-crt-heap-l1-1-0.dll
 0000:fffd9000       .debug$S                   0000000180000000     ucrt:api-ms-win-crt-heap-l1-1-0.dll
 0000:fffd9000       .debug$S                   0000000180000000     ucrt:api-ms-win-crt-runtime-l1-1-0.dll
 0000:fffd9000       .debug$S                   0000000180000000     ucrt:api-ms-win-crt-runtime-l1-1-0.dll
 0000:fffd9000       .debug$S                   0000000180000000     ucrt:api-ms-win-crt-runtime-l1-1-0.dll
 0000:fffd9000       .debug$S                   0000000180000000     ucrt:api-ms-win-crt-runtime-l1-1-0.dll
 0000:fffd9000       .debug$S                   0000000180000000     ucrt:api-ms-win-crt-runtime-l1-1-0.dll
 0000:fffd9000       .debug$S                   0000000180000000     ucrt:api-ms-win-crt-runtime-l1-1-0.dll
 0000:fffd9000       .debug$S                   0000000180000000     ucrt:api-ms-win-crt-runtime-l1-1-0.dll
 0000:fffd9000       .debug$S                   0000000180000000     ucrt:api-ms-win-crt-runtime-l1-1-0.dll
 0000:fffd9000       .debug$S                   0000000180000000     ucrt:api-ms-win-crt-runtime-l1-1-0.dll
 0000:fffd9000       .debug$S                   0000000180000000     ucrt:api-ms-win-crt-runtime-l1-1-0.dll
 0000:fffd9000       .debug$S                   0000000180000000     ucrt:api-ms-win-crt-runtime-l1-1-0.dll
 0000:fffd9000       .debug$S                   0000000180000000     ucrt:api-ms-win-crt-runtime-l1-1-0.dll
 0000:fffd9000       .debug$S                   0000000180000000     ucrt:api-ms-win-crt-runtime-l1-1-0.dll
 0000:fffd9000       .debug$S                   0000000180000000     ucrt:api-ms-win-crt-runtime-l1-1-0.dll
 0000:fffd9000       .debug$S                   0000000180000000     ucrt:api-ms-win-crt-runtime-l1-1-0.dll
 0000:fffd9000       .debug$S                   0000000180000000     ucrt:api-ms-win-crt-runtime-l1-1-0.dll
 0000:fffd9000       .debug$S                   0000000180000000     ucrt:api-ms-win-crt-stdio-l1-1-0.dll
 0000:fffd9000       .debug$S                   0000000180000000     ucrt:api-ms-win-crt-stdio-l1-1-0.dll
 0000:fffd9000       .debug$S                   0000000180000000     ucrt:api-ms-win-crt-stdio-l1-1-0.dll
 0000:fffd9000       .debug$S                   0000000180000000     ucrt:api-ms-win-crt-stdio-l1-1-0.dll
 0000:fffd9000       .debug$S                   0000000180000000     ucrt:api-ms-win-crt-stdio-l1-1-0.dll
 0000:fffd9000       .debug$S                   0000000180000000     ucrt:api-ms-win-crt-stdio-l1-1-0.dll
 0000:fffd9000       .debug$S                   0000000180000000     ucrt:api-ms-win-crt-stdio-l1-1-0.dll
 0000:fffd9000       .debug$S                   0000000180000000     ucrt:api-ms-win-crt-stdio-l1-1-0.dll
 0000:fffd9000       .debug$S                   0000000180000000     ucrt:api-ms-win-crt-stdio-l1-1-0.dll
 0000:fffd9000       .debug$S                   0000000180000000     ucrt:api-ms-win-crt-stdio-l1-1-0.dll
 0000:fffd9000       .debug$S                   0000000180000000     ucrt:api-ms-win-crt-string-l1-1-0.dll
 0000:fffd9000       .debug$S                   0000000180000000     ucrt:api-ms-win-crt-string-l1-1-0.dll
 0000:fffd9000       .debug$S                   0000000180000000     ucrt:api-ms-win-crt-string-l1-1-0.dll
 0000:fffd9000       .debug$S                   0000000180000000     ucrt:api-ms-win-crt-string-l1-1-0.dll
 0000:fffd9000       .debug$S                   0000000180000000     ucrt:api-ms-win-crt-string-l1-1-0.dll
 0000:fffd9000       .debug$S                   0000000180000000     ucrt:api-ms-win-crt-string-l1-1-0.dll
 0000:fffd9000       .debug$S                   0000000180000000     ucrt:api-ms-win-crt-string-l1-1-0.dll
 0000:fffd9000       .debug$S                   0000000180000000     ucrt:api-ms-win-crt-string-l1-1-0.dll
 0000:fffd9000       .debug$S                   0000000180000000     kernel32:KERNEL32.dll
 0000:fffd9000       .debug$S                   0000000180000000     kernel32:KERNEL32.dll
 0000:fffd9000       .debug$S                   0000000180000000     kernel32:KERNEL32.dll
 0000:fffd9000       .debug$S                   0000000180000000     kernel32:KERNEL32.dll
 0000:fffd9000       .debug$S                   0000000180000000     kernel32:KERNEL32.dll
 0000:fffd9000       .debug$S                   0000000180000000     kernel32:KERNEL32.dll
 0000:fffd9000       .debug$S                   0000000180000000     kernel32:KERNEL32.dll
 0000:fffd9000       .debug$S                   0000000180000000     kernel32:KERNEL32.dll
 0000:fffd9000       .debug$S                   0000000180000000     kernel32:KERNEL32.dll
 0000:fffd9000       .debug$S                   0000000180000000     kernel32:KERNEL32.dll
 0000:fffd9000       .debug$S                   0000000180000000     kernel32:KERNEL32.dll
 0000:fffd9000       .debug$S                   0000000180000000     kernel32:KERNEL32.dll
 0000:fffd9000       .debug$S                   0000000180000000     kernel32:KERNEL32.dll
 0000:fffd9000       .debug$S                   0000000180000000     kernel32:KERNEL32.dll
 0000:fffd9000       .debug$S                   0000000180000000     kernel32:KERNEL32.dll
 0000:fffd9000       .debug$S                   0000000180000000     kernel32:KERNEL32.dll
 0000:fffd9000       .debug$S                   0000000180000000     kernel32:KERNEL32.dll
 0000:fffd9000       .debug$S                   0000000180000000     kernel32:KERNEL32.dll
 0000:fffd9000       .debug$S                   0000000180000000     kernel32:KERNEL32.dll
 0000:fffd9000       .debug$S                   0000000180000000     kernel32:KERNEL32.dll
 0000:fffd9000       .debug$S                   0000000180000000     kernel32:KERNEL32.dll
 0000:fffd9000       .debug$S                   0000000180000000     kernel32:KERNEL32.dll
 0000:fffd9000       .debug$S                   0000000180000000     kernel32:KERNEL32.dll
 0000:fffd9000       .debug$S                   0000000180000000     kernel32:KERNEL32.dll
 0000:fffd9000       .debug$S                   0000000180000000     kernel32:KERNEL32.dll
 0000:fffd9000       .debug$S                   0000000180000000     kernel32:KERNEL32.dll
 0000:fffd9000       .debug$S                   0000000180000000     kernel32:KERNEL32.dll
 0000:fffd9000       .debug$S                   0000000180000000     kernel32:KERNEL32.dll
 0001:00000000       default_heap_object_callback 0000000180001000 f   libHeap.obj
 0001:000013b8       addRefToVerify             00000001800023b8 f   libHeap.obj
 0001:00001424       agentThreadWrapper         0000000180002424 f   libHeap.obj
 0001:00001590       default_object_free        0000000180002590 f   libHeap.obj
 0001:0000162c       file_basename              000000018000262c f   libHeap.obj
 0001:000016a0       klass_tag_test_callback    00000001800026a0 f   libHeap.obj
 0001:00001ca8       object_free_count_callback 0000000180002ca8 f   libHeap.obj
 0001:00001d24       simple_heap_root_callback  0000000180002d24 f   libHeap.obj
 0001:00001d80       simple_object_ref_callback 0000000180002d80 f   libHeap.obj
 0001:00001dd4       simple_stack_ref_callback  0000000180002dd4 f   libHeap.obj
 0001:00001e50       startAgentThreadWrapper    0000000180002e50 f   libHeap.obj
 0001:00002190       syncDebuggeeStatus         0000000180003190 f   libHeap.obj
 0001:00002328       tagged_object_count_callback 0000000180003328 f   libHeap.obj
 0001:00002380       total_object_count_callback 0000000180003380 f   libHeap.obj
 0001:000024e0       capture_previous_context   00000001800034e0 f   MSVCRT:gs_report.obj
 0001:00002554       ?__scrt_initialize_thread_safe_statics@@YAHXZ 0000000180003554 f   MSVCRT:thread_safe_statics.obj
 0001:00002624       ?__scrt_uninitialize_thread_safe_statics@@YAXXZ 0000000180003624 f   MSVCRT:thread_safe_statics.obj
 0001:000026d0       $$000000                   00000001800036d0     MSVCRT:amdsecgs.obj
 0001:00002700       ?dllmain_crt_dispatch@@YAHQEAUHINSTANCE__@@KQEAX@Z 0000000180003700 f   MSVCRT:dll_dllmain.obj
 0001:00002750       ?dllmain_crt_process_attach@@YAHQEAUHINSTANCE__@@QEAX@Z 0000000180003750 f   MSVCRT:dll_dllmain.obj
 0001:00002868       ?dllmain_crt_process_detach@@YAH_N@Z 0000000180003868 f   MSVCRT:dll_dllmain.obj
 0001:000028ec       ?dllmain_dispatch@@YAHQEAUHINSTANCE__@@KQEAX@Z 00000001800038ec f   MSVCRT:dll_dllmain.obj
 0001:00003300       $$000000                   0000000180004300     MSVCRT:guard_dispatch.obj
 0001:00003320       $$000000                   0000000180004320     MSVCRT:guard_xfg_dispatch.obj
 0001:00003336       ?fin$0@?0??dllmain_crt_process_attach@@YAHQEAUHINSTANCE__@@QEAX@Z@4HA 0000000180004336 f   MSVCRT:dll_dllmain.obj
 0001:0000334d       ?fin$0@?0??dllmain_crt_process_detach@@YAH_N@Z@4HA 000000018000434d f   MSVCRT:dll_dllmain.obj
 0001:00003366       ?fin$1@?0??dllmain_crt_process_detach@@YAH_N@Z@4HA 0000000180004366 f   MSVCRT:dll_dllmain.obj
 0001:0000337a       ?filt$0@?0??dllmain_dispatch@@YAHQEAUHINSTANCE__@@KQEAX@Z@4HA 000000018000437a f   MSVCRT:dll_dllmain.obj
 0001:000033b0       __scrt_is_nonwritable_in_current_image$filt$0 00000001800043b0 f   MSVCRT:utility.obj
 0002:000001f8       ?__scrt_initialize_tss_var@@3P6AHXZEA 00000001800051f8     MSVCRT:thread_safe_statics.obj
 0002:00000320       ?opcLengths@@3QBEB         0000000180005320     libHeap.obj
 0002:00001ce8       GS_ExceptionPointers       0000000180006ce8     MSVCRT:gs_report.obj
 0002:00002390       $unwind$fprintf            0000000180007390     libHeap.obj
 0002:0000239c       $unwind$printf             000000018000739c     libHeap.obj
 0002:000023a8       $unwind$?NewObject@JNIEnv_@@QEAAPEAV_jobject@@PEAV_jclass@@PEAU_jmethodID@@ZZ 00000001800073a8     libHeap.obj
 0002:000023a8       $unwind$nsk_lcomplain      00000001800073a8     libHeap.obj
 0002:000023a8       $unwind$nsk_ldisplay       00000001800073a8     libHeap.obj
 0002:000023b0       $unwind$klass_tag_test_callback 00000001800073b0     libHeap.obj
 0002:000023b0       $unwind$nsk_lvdisplay      00000001800073b0     libHeap.obj
 0002:000023b0       $unwind$simple_heap_root_callback 00000001800073b0     libHeap.obj
 0002:000023b0       $unwind$_RTC_Initialize    00000001800073b0     MSVCRT:initsect.obj
 0002:000023b0       $unwind$_RTC_Terminate     00000001800073b0     MSVCRT:initsect.obj
 0002:000023b0       $unwind$?__scrt_initialize_thread_safe_statics@@YAHXZ 00000001800073b0     MSVCRT:thread_safe_statics.obj
 0002:000023bc       $unwind$nsk_lvcomplain     00000001800073bc     libHeap.obj
 0002:000023d4       $unwind$nsk_ltrace         00000001800073d4     libHeap.obj
 0002:000023d4       $unwind$__report_gsfailure 00000001800073d4     MSVCRT:gs_report.obj
 0002:000023dc       $unwind$Java_nsk_share_jvmti_unit_Heap_getObjectSize 00000001800073dc     libHeap.obj
 0002:000023dc       $unwind$Java_nsk_share_jvmti_unit_Heap_getTag0 00000001800073dc     libHeap.obj
 0002:000023dc       $unwind$Java_nsk_share_jvmti_unit_Heap_iterateOverHeap0 00000001800073dc     libHeap.obj
 0002:000023dc       $unwind$Java_nsk_share_jvmti_unit_Heap_iterateOverObjectsReachableFromObject0 00000001800073dc     libHeap.obj
 0002:000023dc       $unwind$nsk_lvtrace        00000001800073dc     libHeap.obj
 0002:000023dc       $unwind$simple_object_ref_callback 00000001800073dc     libHeap.obj
 0002:000023dc       $unwind$simple_stack_ref_callback 00000001800073dc     libHeap.obj
 0002:000023dc       $unwind$tagged_object_count_callback 00000001800073dc     libHeap.obj
 0002:000023dc       $unwind$total_object_count_callback 00000001800073dc     libHeap.obj
 0002:000023dc       $unwind$__raise_securityfailure 00000001800073dc     MSVCRT:gs_report.obj
 0002:000023dc       $unwind$__scrt_initialize_crt 00000001800073dc     MSVCRT:utility.obj
 0002:000023dc       $unwind$__scrt_initialize_onexit_tables 00000001800073dc     MSVCRT:utility.obj
 0002:000023dc       $unwind$__scrt_release_startup_lock 00000001800073dc     MSVCRT:utility.obj
 0002:000023dc       $unwind$__scrt_uninitialize_crt 00000001800073dc     MSVCRT:utility.obj
 0002:000023dc       $unwind$_onexit            00000001800073dc     MSVCRT:utility.obj
 0002:000023e4       $unwind$nsk_lverify        00000001800073e4     libHeap.obj
 0002:000023f4       $unwind$nsk_vprintf        00000001800073f4     libHeap.obj
 0002:00002404       $unwind$nsk_printf         0000000180007404     libHeap.obj
 0002:0000240c       $unwind$?nsk_jni_lverify@@YAHHPEAUJNIEnv_@@HQEBDH1ZZ 000000018000740c     libHeap.obj
 0002:00002420       $unwind$?nsk_jni_check_exception@@YAHPEAUJNIEnv_@@QEBDH@Z 0000000180007420     libHeap.obj
 0002:0000243c       $unwind$Java_nsk_jvmti_unit_FollowReferences_FollowRefObjects_resetTags 000000018000743c     libHeap.obj
 0002:0000243c       $unwind$addRefToVerify     000000018000743c     libHeap.obj
 0002:0000243c       $unwind$default_heap_object_callback 000000018000743c     libHeap.obj
 0002:0000243c       $unwind$default_object_free 000000018000743c     libHeap.obj
 0002:0000243c       $unwind$nsk_jvmti_resetAgentData 000000018000743c     libHeap.obj
 0002:0000243c       $unwind$nsk_jvmti_setFailStatus 000000018000743c     libHeap.obj
 0002:0000243c       $unwind$object_free_count_callback 000000018000743c     libHeap.obj
 0002:0000243c       $unwind$__scrt_initialize_default_local_stdio_options 000000018000743c     MSVCRT:default_local_stdio_options.obj
 0002:0000243c       $unwind$?dllmain_crt_dispatch@@YAHQEAUHINSTANCE__@@KQEAX@Z 000000018000743c     MSVCRT:dll_dllmain.obj
 0002:0000243c       $unwind$DllMain            000000018000743c     MSVCRT:dll_dllmain_stub.obj
 0002:0000243c       $unwind$__GSHandlerCheck   000000018000743c     MSVCRT:gshandler.obj
 0002:0000243c       $unwind$?__scrt_uninitialize_thread_safe_statics@@YAXXZ 000000018000743c     MSVCRT:thread_safe_statics.obj
 0002:0000243c       $unwind$__scrt_acquire_startup_lock 000000018000743c     MSVCRT:utility.obj
 0002:0000243c       $unwind$__scrt_dllmain_after_initialize_c 000000018000743c     MSVCRT:utility.obj
 0002:0000243c       $unwind$__scrt_dllmain_before_initialize_c 000000018000743c     MSVCRT:utility.obj
 0002:0000243c       $unwind$__scrt_dllmain_crt_thread_attach 000000018000743c     MSVCRT:utility.obj
 0002:0000243c       $unwind$__scrt_dllmain_crt_thread_detach 000000018000743c     MSVCRT:utility.obj
 0002:0000243c       $unwind$__scrt_dllmain_uninitialize_c 000000018000743c     MSVCRT:utility.obj
 0002:0000243c       $unwind$__scrt_dllmain_uninitialize_critical 000000018000743c     MSVCRT:utility.obj
 0002:0000243c       $unwind$atexit             000000018000743c     MSVCRT:utility.obj
 0002:00002444       $unwind$nsk_jvmti_lverify  0000000180007444     libHeap.obj
 0002:00002458       $unwind$exitOnError        0000000180007458     libHeap.obj
 0002:00002468       $unwind$Java_nsk_share_jvmti_ArgumentHandler_getAgentOptionsString 0000000180007468     libHeap.obj
 0002:0000247c       $unwind$Java_nsk_jvmti_unit_FollowReferences_FollowRefObjects_getTag 000000018000747c     libHeap.obj
 0002:0000247c       $unwind$Java_nsk_share_jvmti_DebugeeClass_checkStatus 000000018000747c     libHeap.obj
 0002:0000247c       $unwind$agentThreadWrapper 000000018000747c     libHeap.obj
 0002:0000248c       $unwind$startAgentThreadWrapper 000000018000748c     libHeap.obj
 0002:000024a8       $unwind$syncDebuggeeStatus 00000001800074a8     libHeap.obj
 0002:000024a8       $unwind$__scrt_dllmain_exception_filter 00000001800074a8     MSVCRT:utility.obj
 0002:000024bc       $unwind$Java_nsk_share_jvmti_DebugeeClass_resetAgentData 00000001800074bc     libHeap.obj
 0002:000024c4       $unwind$MA_checkStatus     00000001800074c4     libHeap.obj
 0002:000024d8       $unwind$Java_nsk_jvmti_unit_FollowReferences_FollowRefObjects_setTag 00000001800074d8     libHeap.obj
 0002:000024f0       $unwind$Java_nsk_jvmti_unit_FollowReferences_FollowRefObjects_addRefToVerify 00000001800074f0     libHeap.obj
 0002:0000250c       $unwind$Agent_Initialize   000000018000750c     libHeap.obj
 0002:00002520       $unwind$Java_nsk_share_jvmti_unit_Heap_iterateOverInstancesOfClass0 0000000180007520     libHeap.obj
 0002:0000252c       $unwind$Java_nsk_share_jvmti_unit_Heap_iterateOverReachableObjects0 000000018000752c     libHeap.obj
 0002:00002534       $unwind$Java_nsk_share_jvmti_unit_Heap_getObjectsWithTags 0000000180007534     libHeap.obj
 0002:00002548       $unwind$capture_previous_context 0000000180007548     MSVCRT:gs_report.obj
 0002:00002554       $unwind$__GSHandlerCheckCommon 0000000180007554     MSVCRT:gshandler.obj
 0002:00002560       $xdatasym                  0000000180007560     MSVCRT:amdsecgs.obj
 0002:00002564       $unwind$?dllmain_crt_process_attach@@YAHQEAUHINSTANCE__@@QEAX@Z 0000000180007564     MSVCRT:dll_dllmain.obj
 0002:000025a0       $unwind$?fin$0@?0??dllmain_crt_process_attach@@YAHQEAUHINSTANCE__@@QEAX@Z@4HA 00000001800075a0     MSVCRT:dll_dllmain.obj
 0002:000025a0       $unwind$?fin$0@?0??dllmain_crt_process_detach@@YAH_N@Z@4HA 00000001800075a0     MSVCRT:dll_dllmain.obj
 0002:000025a0       $unwind$?fin$1@?0??dllmain_crt_process_detach@@YAH_N@Z@4HA 00000001800075a0     MSVCRT:dll_dllmain.obj
 0002:000025a8       $unwind$?dllmain_crt_process_detach@@YAH_N@Z 00000001800075a8     MSVCRT:dll_dllmain.obj
 0002:000025fc       $unwind$?dllmain_dispatch@@YAHQEAUHINSTANCE__@@KQEAX@Z 00000001800075fc     MSVCRT:dll_dllmain.obj
 0002:00002624       $unwind$?filt$0@?0??dllmain_dispatch@@YAHQEAUHINSTANCE__@@KQEAX@Z@4HA 0000000180007624     MSVCRT:dll_dllmain.obj
 0002:0000262c       $unwind$_DllMainCRTStartup 000000018000762c     MSVCRT:dll_dllmain.obj
 0002:0000263c       $unwind$__scrt_is_nonwritable_in_current_image 000000018000763c     MSVCRT:utility.obj
 0002:0000265c       $unwind$__scrt_is_nonwritable_in_current_image$filt$0 000000018000765c     MSVCRT:utility.obj
 0002:00002664       $unwind$__scrt_fastfail    0000000180007664     MSVCRT:utility_desktop.obj
 0002:00002674       $unwind$__security_init_cookie 0000000180007674     MSVCRT:gs_support.obj
 0002:00002680       $unwind$__isa_available_init 0000000180007680     MSVCRT:cpu_disp.obj
 0002:00002690       $xdatasym                  0000000180007690     MSVCRT:guard_dispatch.obj
 0002:00002698       $xdatasym                  0000000180007698     MSVCRT:guard_xfg_dispatch.obj
 0002:000026a0       .edata                     00000001800076a0     Heap.exp
 0002:000026c8       rgpv                       00000001800076c8     Heap.exp
 0002:00002758       rgszName                   0000000180007758     Heap.exp
 0002:000027e8       rgwOrd                     00000001800077e8     Heap.exp
 0002:00002830       szName                     0000000180007830     Heap.exp
 0002:00002839       $N00001                    0000000180007839     Heap.exp
 0002:00002848       $N00002                    0000000180007848     Heap.exp
 0002:00002855       $N00003                    0000000180007855     Heap.exp
 0002:0000289a       $N00004                    000000018000789a     Heap.exp
 0002:000028d7       $N00005                    00000001800078d7     Heap.exp
 0002:0000291f       $N00006                    000000018000791f     Heap.exp
 0002:0000295f       $N00007                    000000018000795f     Heap.exp
 0002:0000299c       $N00008                    000000018000799c     Heap.exp
 0002:000029d7       $N00009                    00000001800079d7     Heap.exp
 0002:00002a05       $N00010                    0000000180007a05     Heap.exp
 0002:00002a36       $N00011                    0000000180007a36     Heap.exp
 0002:00002a65       $N00012                    0000000180007a65     Heap.exp
 0002:00002a94       $N00013                    0000000180007a94     Heap.exp
 0002:00002ac9       $N00014                    0000000180007ac9     Heap.exp
 0002:00002af7       $N00015                    0000000180007af7     Heap.exp
 0002:00002b29       $N00016                    0000000180007b29     Heap.exp
 0002:00002b56       $N00017                    0000000180007b56     Heap.exp
 0002:00002b88       $N00018                    0000000180007b88     Heap.exp
 0002:00002baf       $N00019                    0000000180007baf     Heap.exp
 0002:00002bdf       $N00020                    0000000180007bdf     Heap.exp
 0002:00002c1b       $N00021                    0000000180007c1b     Heap.exp
 0002:00002c61       $N00022                    0000000180007c61     Heap.exp
 0002:00002c9d       $N00023                    0000000180007c9d     Heap.exp
 0002:00002cc9       $N00024                    0000000180007cc9     Heap.exp
 0002:00002cf6       $N00025                    0000000180007cf6     Heap.exp
 0002:00002d29       $N00026                    0000000180007d29     Heap.exp
 0002:00002d60       $N00027                    0000000180007d60     Heap.exp
 0002:00002d95       $N00028                    0000000180007d95     Heap.exp
 0002:00002dc9       $N00029                    0000000180007dc9     Heap.exp
 0002:00002dfc       $N00030                    0000000180007dfc     Heap.exp
 0002:00002e23       $N00031                    0000000180007e23     Heap.exp
 0002:00002e5f       $N00032                    0000000180007e5f     Heap.exp
 0002:00002e9a       $N00033                    0000000180007e9a     Heap.exp
 0002:00002ec4       $N00034                    0000000180007ec4     Heap.exp
 0002:00002ef3       $N00035                    0000000180007ef3     Heap.exp
 0002:00002f26       $N00036                    0000000180007f26     Heap.exp
 0002:0000335a       .idata$6                   000000018000835a     kernel32:KERNEL32.dll
 0002:000033be       .idata$6                   00000001800083be     vcruntime:VCRUNTIME140.dll
 0002:00003532       .idata$6                   0000000180008532     ucrt:api-ms-win-crt-heap-l1-1-0.dll
 0002:00003552       .idata$6                   0000000180008552     ucrt:api-ms-win-crt-runtime-l1-1-0.dll
 0002:00003574       .idata$6                   0000000180008574     ucrt:api-ms-win-crt-stdio-l1-1-0.dll
 0002:00003594       .idata$6                   0000000180008594     ucrt:api-ms-win-crt-string-l1-1-0.dll
 0003:00000000       ?codeAttributeName@@3PEBDEB 0000000180009000     libHeap.obj
 0003:00000008       ?lineNumberAttributeName@@3PEBDEB 0000000180009008     libHeap.obj
 0003:00000010       ?localVarAttributeName@@3PEBDEB 0000000180009010     libHeap.obj
 0003:00000018       ?localVarTypeAttributeName@@3PEBDEB 0000000180009018     libHeap.obj
 0003:00000020       ?stackMapAttributeName@@3PEBDEB 0000000180009020     libHeap.obj
 0003:00000028       ?callBytes@@3PAEA          0000000180009028     libHeap.obj
 0003:0000002c       ?allocBytes@@3PAEA         000000018000902c     libHeap.obj
 0003:00000030       heap_object_callback       0000000180009030     libHeap.obj
 0003:0001aad4       redefineAttempted          0000000180023ad4     libHeap.obj
 0003:0001aad8       nsk_context                0000000180023ad8     libHeap.obj
 0003:0001aae4       redefineSucceed            0000000180023ae4     libHeap.obj
 0003:0001aae8       agentFailed                0000000180023ae8     libHeap.obj
 0003:0001aaec       currentAgentStatus         0000000180023aec     libHeap.obj
 0003:0001aaf0       context                    0000000180023af0     libHeap.obj
 0003:0001aba8       agentThread                0000000180023ba8     libHeap.obj
 0003:0001abb0       agentThreadProc            0000000180023bb0     libHeap.obj
 0003:0001abb8       agentThreadArg             0000000180023bb8     libHeap.obj
 0003:0001abc0       agent_data                 0000000180023bc0     libHeap.obj
 0003:0001abd0       jvmti_env                  0000000180023bd0     libHeap.obj
 0003:0001abd8       jvm                        0000000180023bd8     libHeap.obj
 0003:0001abe0       jni_env                    0000000180023be0     libHeap.obj
 0003:0001abe8       checkStatus_func           0000000180023be8     libHeap.obj
 0003:0001abf0       ?codeAttributeIndex@@3GA   0000000180023bf0     libHeap.obj
 0003:0001abf2       user_data_error_flag       0000000180023bf2     libHeap.obj
 0003:0001abf4       ?lineNumberAttributeIndex@@3GA 0000000180023bf4     libHeap.obj
 0003:0001abf8       ?localVarAttributeIndex@@3GA 0000000180023bf8     libHeap.obj
 0003:0001abfc       ?localVarTypeAttributeIndex@@3GA 0000000180023bfc     libHeap.obj
 0003:0001ac00       ?stackMapAttributeIndex@@3GA 0000000180023c00     libHeap.obj
 0003:0001ac04       ?stackFrameOffset@@3GA     0000000180023c04     libHeap.obj
 0003:0001ac08       ?mode@@3HA                 0000000180023c08     libHeap.obj
 0003:0001ac0c       ?constantPoolSize@@3GA     0000000180023c0c     libHeap.obj
 0003:0001ac10       ?orig@@3PEBEEB             0000000180023c10     libHeap.obj
 0003:0001ac18       ?gen@@3PEAEEA              0000000180023c18     libHeap.obj
 0003:0001ac20       ?inputPos@@3PEAEEA         0000000180023c20     libHeap.obj
 0003:0001ac28       ?endPos@@3PEBEEB           0000000180023c28     libHeap.obj
 0003:0001ac30       ?genPos@@3PEAEEA           0000000180023c30     libHeap.obj
 0003:0001ac38       ?markPos@@3PEAEEA          0000000180023c38     libHeap.obj
 0003:0001ac40       ?constantPool@@3PEAPEADEA  0000000180023c40     libHeap.obj
 0003:0001ac48       ?constantPoolCount@@3GA    0000000180023c48     libHeap.obj
 0003:0001ac4c       ?zeroBytes@@3PAEA          0000000180023c4c     libHeap.obj
 0003:0001ac50       ?codeLength@@3IA           0000000180023c50     libHeap.obj
 0003:0001ac54       dummy_user_data            0000000180023c54     libHeap.obj
 0003:0001ac58       ?map@@3PEAIEA              0000000180023c58     libHeap.obj
 0003:0001ac60       ?widening@@3PEACEA         0000000180023c60     libHeap.obj
 0003:0001ac68       jvmti                      0000000180023c68     libHeap.obj
 0003:0001ac70       object_free_callback       0000000180023c70     libHeap.obj
 0003:0001ac78       heap_root_callback         0000000180023c78     libHeap.obj
 0003:0001ac80       stack_ref_callback         0000000180023c80     libHeap.obj
 0003:0001ac88       object_ref_callback        0000000180023c88     libHeap.obj
 0003:0001ac90       object_results_ref         0000000180023c90     libHeap.obj
 0003:0001ac98       tag_results_ref            0000000180023c98     libHeap.obj
 0003:0001aca0       object_count               0000000180023ca0     libHeap.obj
 0003:0001aca4       object_free_count          0000000180023ca4     libHeap.obj
 0003:0001acb0       GS_ExceptionRecord         0000000180023cb0     MSVCRT:gs_report.obj
 0003:0001ad50       GS_ContextRecord           0000000180023d50     MSVCRT:gs_report.obj
 0003:0001b220       ?g_tss_cv@@3U_RTL_CONDITION_VARIABLE@@A 0000000180024220     MSVCRT:thread_safe_statics.obj
 0003:0001b228       ?g_tss_event@@3PEAXEA      0000000180024228     MSVCRT:thread_safe_statics.obj
 0003:0001b230       ?g_tss_mutex@@3U_RTL_CRITICAL_SECTION@@A 0000000180024230     MSVCRT:thread_safe_statics.obj
 0003:0001b258       ?g_sleep_condition_variable_cs@@3P6AHPEAU_RTL_CONDITION_VARIABLE@@PEAU_RTL_CRITICAL_SECTION@@K@ZEA 0000000180024258     MSVCRT:thread_safe_statics.obj
 0003:0001b260       ?g_wake_all_condition_variable@@3P6AXPEAU_RTL_CONDITION_VARIABLE@@@ZEA 0000000180024260     MSVCRT:thread_safe_statics.obj
 0003:0001b26c       ?__proc_attached@@3HA      000000018002426c     MSVCRT:dll_dllmain.obj
 0003:0001b280       ?is_initialized_as_dll@@3_NA 0000000180024280     MSVCRT:utility.obj
 0003:0001b281       ?module_local_atexit_table_initialized@@3_NA 0000000180024281     MSVCRT:utility.obj
 0003:0001b288       ?module_local_atexit_table@@3U_onexit_table_t@@A 0000000180024288     MSVCRT:utility.obj
 0003:0001b2a0       ?module_local_at_quick_exit_table@@3U_onexit_table_t@@A 00000001800242a0     MSVCRT:utility.obj
